:100000000C9437010C9454010C9454010C94540139
:100010000C9454010C9454010C9454010C9454010C
:100020000C9454010C9454010C94D81C0C94AA1DEB
:100030000C94CA170C9454010C9454010C94540160
:100040000C9454010C9454010C9454010C945401DC
:100050000C9454010C9452180C9454010C945401B7
:100060000C9454010C9454010C9454010C945401BC
:100070000C9454010C9454010C9454010C945401AC
:100080000C9454010C9454010C9454010C9454019C
:100090000C9454010C9454010C9454010C9454018C
:1000A0000C9454010C9454010C9454010A040A0455
:1000B000360436049E04BC04D405D405C704600588
:1000C00071057105171E3E1E361F3E1E361F8A1E05
:1000D000AD1E361F041F131F1E001F00200021002D
:1000E000220014001A000800150017001403320043
:1000F000780035006B0065007900700061006400D5
:10010000000022034A006F006E0061007400680066
:1001100061006E002000430061006D006500720008
:100120006F006E0000000403090409023B00020195
:1001300000A0FA09040000010301010009211101D6
:1001400000012240000705810308000109040100A5
:10015000010300000009211101000122B60007057A
:1001600082032000011201000200000008EDFE20C1
:100170002001000102000105010902A10185020917
:1001800001A1000509190129081500250195087527
:100190000181020501093009311581257F9502751C
:1001A00008810609381581257F95017508810605A6
:1001B0000C0A38021581257F950175088106C0C09B
:1001C00005010980A101850319012AB7001501263F
:1001D000B700950175108100C0050C0901A10185CA
:1001E0000419012AA002150126A0029501751081AB
:1001F00000C005010906A1018506050719E029E7E8
:10020000150025019508750181020507190029EFE0
:100210001500250195F075018102050819012905D0
:10022000950575019102950175039101C0050109BC
:1002300006A101050719E029E715002501950875B4
:100240000181029501750881010507190029FF1533
:100250000026FF009506750881000508190129058B
:10026000950575019102950175039101C000112456
:100270001FBECFEFDAE0DEBFCDBF11E0A0E0B1E0FE
:10028000E2EDFFE302C005900D92A238B107D9F765
:1002900022E0A2E8B1E001C01D92A737B207E1F762
:1002A0000E9492110C94E71F0C9400000E9475109C
:1002B000509A259A269A089581E0089581E008953C
:1002C0000C945E0108950C9462011F93CF93DF9309
:1002D00000D000D01F92CDB7DEB749835A836B831D
:1002E0003091850189819A81311114C0662359F0BA
:1002F000222349F00E941308182F682F89819A81C0
:100300000E94BA0703C00E94E607182F69817A810C
:10031000812F04C00E94130869817A810F900F9089
:100320000F900F900F90DF91CF911F910C94340F8D
:10033000FC01262F408151816281738184810C945C
:10034000650181E00895CF93DF93EC0160E00E94A6
:100350009801BE01DF91CF910C9463010C9456017A
:100360000C94731008950E9464060E94B2012FEF4E
:1003700084E39CE0215080409040E1F700C0000001
:100380000C9478180F931F93CF93DF938C0161E047
:100390000E949801EC01B8010E9460018823F1F1EC
:1003A000B801CE010E9414168823C1F1B801CE0114
:1003B0000E942814882391F1B801CE010E94701583
:1003C000882361F1F8018281882309F1CB358DE51D
:1003D000D807C1F050F4C115FCE5DF0781F0CF3D2F
:1003E000DC45A9F40E944A0D19C0CC35EDE5DE07C5
:1003F00061F0CD35DD4559F40E948D0C08C00E9496
:10040000B3010CC00E94960C02C00E94990CC80156
:10041000DF91CF911F910F910C945C0180E0DF91EF
:10042000CF911F910F9108950E94AB170C942D024C
:100430000E9430020C94B11708950C941C0281E0C4
:1004400008950C941F020895CF93C82F0E941D0297
:100450008C2F0E942102CF91089580E00C942402F9
:100460000E9470160C9424020E94701690918401D0
:10047000891721F0809384010C9424020895CF936E
:10048000DF93CDB7DEB72B970FB6F894DEBF0FBE64
:10049000CDBF4F83588769877A878B8761110E9408
:1004A000D90B9E012F5F3F4F86E0F90111928A958B
:1004B000E9F785E0FE013796D90101900D928A9502
:1004C000E1F789819A814C815D81452B31F09F3F15
:1004D00031F491E08F3F19F403C091E001C090E046
:1004E00090FF09C049815A816B817C818D819E81F9
:1004F0000E94FA0A05C0C9010E94A1018111F2CF30
:100500002B960FB6F894DEBF0FBECDBFDF91CF9113
:100510000895FC01808191810E9455080895CF9330
:10052000882309F4A4C0C82F8238C1F40E94701631
:1005300081FD9DC069E380910201909103010E94B9
:1005400066170E94FB0B2FEF81EE94E02150804054
:100550009040E1F700C0000069E319C0833801F55D
:100560000E94701680FD83C063E580910201909126
:1005700003010E9466170E94FB0B2FEF81EE94E0AF
:10058000215080409040E1F700C0000063E5809179
:100590000201909103010E947117CF910C94FB0B03
:1005A0008438C1F40E94701682FD61C067E48091B6
:1005B0000201909103010E9466170E94FB0B2FEF2E
:1005C00081EE94E0215080409040E1F700C00000AF
:1005D00067E4DDCF8CEF8C0F813AD0F46C2F8091E3
:1005E0000201909103010E94E616882349F06C2FC6
:1005F00080910201909103010E9471170E94FB0BF0
:100600006C2F80910201909103010E946617C5CF63
:1006100080E28C0F883048F4C77081E001C0880FF9
:10062000CA95EAF70E94BC0BB8CFEBE5EC0FE330BC
:1006300040F4F0E0E95BFE4F808190E0CF910C94B4
:10064000A416E8E5EC0FE73150F4F0E0EE0FFF1FE1
:10065000E75EFE4F80819181CF910C94BA16CD3E1A
:1006600030F08C2F0E941712CF910C94E912CF9189
:100670000895882309F464C0823879F40E947016C2
:1006800081FF5EC069E380910201909103010E94A5
:1006900066170E94FB0B69E310C08338B1F40E9417
:1006A000701680FF4DC063E58091020190910301B7
:1006B0000E9466170E94FB0B63E5809102019091F6
:1006C00003010E9471170C94FB0B843879F40E948B
:1006D000701682FF35C067E480910201909103019A
:1006E0000E9466170E94FB0B67E4E7CF9CEF980F10
:1006F000913A10F4682FE1CF90E2980F983050F4BF
:10070000877091E001C0990F8A95EAF7892F0E94BE
:10071000C20BD9CF9BE5980F933020F480E090E096
:100720000C94A41698E5980F973120F480E090E09F
:100730000C94BA168D3E20F00E9472120C94E912AD
:1007400008951F93CF93DF93182FEB010E948F0220
:10075000209741F08FE99FE00197F1F700C000007A
:100760002197F6CF812FDF91CF911F910C94390300
:10077000893319F060E070E002C060E570E00C942D
:10078000A103882321F00E94BC0B0C94FB0B08955D
:10079000882321F00E94C20B0C94FB0B0895CF928A
:1007A000DF92EF92FF920F931F93CF93DF937C0121
:1007B000D62FC72FFC011281058102950F700E9470
:1007C000B20B8823B9F01123A9F08C2F807F8034DD
:1007D00021F080E28D0F883068F08091610282FD07
:1007E00009C082E00E945B0C0E94B20B91E0D82EFF
:1007F000D92601C0D12CCC2EC2948FE0C8228C2DDA
:1008000090E08C30910508F0CFC1FC01EA5AFF4F0F
:100810000C947E1F8C2F807FCF70882311F0C2959F
:10082000C07F112399F0CC2309F4AAC180E28D0F77
:10083000883010F0D11104C08C2F0E94BC0B03C073
:100840008C2F0E94CC0B0E94FB0B9AC18D2F0E9413
:100850003903CC2309F4A8C180E28D0F883038F128
:10086000DD2329F18C2F0E94D20B24C08C2F807F96
:10087000CF70803211F0C295C07FDD2319F0D130E6
:10088000A1F13DC08091610282FF17C0112349F0A0
:10089000CC2329F08C2F0E94BC0B0E94FB0B80E024
:1008A00070C180E00E943903CC2309F47DC18C2FF4
:1008B0000E94C20B0E94FB0B77C1112371F0002331
:1008C00041F0013031F40E94DC0B8C2B0E94E40BD0
:1008D0006BC10E94DC0B8C2B1DC0002319F0013072
:1008E00009F462C10E94F10B25C0112321F00630EA
:1008F00008F05AC10EC0053008F056C11BC01123C4
:1009000061F0002331F0F701858180FF39C18F70DC
:1009100085838C2F0E94C10347C1002359F0D9332E
:1009200009F03FC1FFEF07EE13E0F1500040104027
:10093000E1F735C18C2F0E94C80336C18C2F8695F4
:100940008695837019F0813061F02EC1112321F05A
:100950008D2F9C2F937002C080E090E00E94A4161F
:100960002BC1112321F08D2F9C2F937002C080E0AA
:1009700090E00E94BA1620C18D2F112319F00E9419
:10098000171202C00E9472120E94E91215C18C2F28
:10099000837009F047C011110BC12D2F22952695A8
:1009A0002770220F220F6D2F6F70862F90E0A0E02E
:1009B000B0E0022E04C0880F991FAA1FBB1F0A9423
:1009C000D2F7D4FF10C04FE050E060E070E004C008
:1009D000440F551F661F771F2A95D2F740955095F3
:1009E0006095709503C040E050E0BA01C695C69589
:1009F000C3708A019B01082B192B2A2B3B2BC901A1
:100A0000B801C23049F058F4C13019F00E94D00644
:100A1000CFC00E94BE06CCC00E94E206C9C00E94A0
:100A2000BC06C6C0112319F08C2F817001C08695B9
:100A3000882309F4BDC02D2F229526952770220FFB
:100A4000220F6D2F6F70862F90E0A0E0B0E0022E95
:100A500004C0880F991FAA1FBB1F0A94D2F7D4FFA6
:100A600010C04FE050E060E070E004C0440F551F3C
:100A7000661F771F2A95D2F740955095609570951F
:100A800003C040E050E0BA01C695C695C3708A0124
:100A90009B01082B192B2A2B3B2BC901B801C23013
:100AA00049F058F4C13019F00E94950781C00E94A6
:100AB00083077EC00E94A7077BC00E94F60678C00D
:100AC000CF70112339F08C2F0E941C078D2F0E94AC
:100AD000C1036EC08D2F0E94C8038C2F0E943D075A
:100AE00067C0D23F21F128F4D03F41F0D13FC1F09F
:100AF00043C0D33F19F1D43F79F03EC0112341F0F8
:100B0000053008F051C08C2F8F710E9462074CC0D5
:100B1000063008F049C0F7CF8091610282FF18C00B
:100B2000112339F08C2F8F710E941C073DC01123B7
:100B3000C9F38C2F8F710E943D0736C0112329F015
:100B40008C2F8F710E9407072FC00E9402072CC0B4
:100B5000112349F0CF718C2F0E941C0763E08C2F6A
:100B60000E94400C21C081E00E945B0C0230E0F04A
:100B700082E00E945B0C18C0112331F0002391F237
:100B80008D2F0E948F0210C0002399F2D93349F4AF
:100B90001FEF27EE33E0115020403040E1F700C056
:100BA00000008D2F0E94390388EF8C0D843020F4D3
:100BB0000E9470160E942402DD20C9F00E94AE0B34
:100BC00080FD15C0F70112820E94A80B0E941C072D
:100BD000C7010E9418060E94A80BDF91CF911F91B8
:100BE0000F91FF90EF90DF90CF900C943D07DF9135
:100BF000CF911F910F91FF90EF90DF90CF900895CC
:100C00000F931F93CF93DF93EC01688179818A81E1
:100C10000E9460088C010E94B9070E94AA06B801D0
:100C2000CE010E94CF03DF91CF911F910F910895C4
:100C3000CF93DF93EC01988189812B813C81232B19
:100C400031F08F3F31F481E09F3F19F403C081E020
:100C500001C080E080FD1DC0CE010E94C201811153
:100C600010C00E94B20B8823A1F08A81882389F0EA
:100C70008091610282FD0DC082E0DF91CF910C94E2
:100C80005B0CCE010E940006CE01DF91CF910C9447
:100C9000A301DF91CF91089580E090E00E94A41617
:100CA00080E090E00E94BA160E94D90B0E94FB0BD4
:100CB0000E941A140C94E912809102019091030190
:100CC0000E947C170C944C060E94C90B0C945C0685
:100CD00092959F70963079F010F4925001C09A501E
:100CE000923068F4803F69F018F4883E40F409C0FF
:100CF000843F29F406C0883E20F0813F11F080E057
:100D0000089581E00895FC01808191810E94550839
:100D10000E9468060895CF93DF9300D000D01F9201
:100D2000CDB7DEB70F900F900F900F900F90DF911F
:100D3000CF910895CF93DF9300D000D000D0CDB7EE
:100D4000DEB726960FB6F894DEBF0FBECDBFDF919B
:100D5000CF910895089508950C94AB060C94AC06B9
:100D60000E94AE0660939401709395018093960162
:100D7000909397010C944C060C94B0060F931F931C
:100D80000091940110919501209196013091970165
:100D9000602B712B822B932B1F910F910C94B0061B
:100DA0000F931F930091940110919501209196014A
:100DB0003091970160237123822393231F910F9118
:100DC0000C94B0060F931F9300919401109195011C
:100DD00020919601309197016027712782279327F0
:100DE0001F910F910C94B0060C94AB060E94F40670
:100DF000609390017093910180939201909393017D
:100E00000C944C0660E070E0CB010C94F6060F9356
:100E10001F9341E050E060E070E08A019B0104C054
:100E2000000F111F221F331F8A95D2F7C901B80185
:100E30001F910F910C94F6060F931F9341E050E021
:100E400060E070E004C0440F551F661F771F8A954D
:100E5000D2F78091900190919101A0919201B0916F
:100E600093018A019B01082B192B2A2B3B2BC901CB
:100E7000B8011F910F910C94F6060F931F9341E058
:100E800050E060E070E004C0440F551F661F771FFC
:100E90008A95D2F740955095609570958091900114
:100EA00090919101A0919201B09193018A019B01CF
:100EB000082319232A233B23C901B8011F910F914D
:100EC0000C94F6060F931F9341E050E060E070E051
:100ED00004C0440F551F661F771F8A95D2F7809173
:100EE000900190919101A0919201B09193018A019A
:100EF0009B01082719272A273B27C901B8011F9101
:100F00000F910C94F6060F931F930091900110918E
:100F100091012091920130919301602B712B822BD2
:100F2000932B1F910F910C94F6060F931F93009132
:100F300090011091910120919201309193016023D1
:100F40007123822393231F910F910C94F6060F9324
:100F50001F93009190011091910120919201309185
:100F6000930160277127822793271F910F910C947B
:100F7000F606089524E0929F900D1124890FE82F22
:100F8000E695E695E695877051E001C0550F8A9584
:100F9000EAF785E0E89FF0011124EA57FE4F20E0D0
:100FA00030E070E04081CB01022E02C0969587951B
:100FB0000A94E2F7817081958427852384278193A1
:100FC0002F5F3F4F2530310569F7089524E0929F48
:100FD000900D1124890F682F669566956695982F58
:100FE000977085E0689FB001112440E050E080E0F8
:100FF000FB01E40FF51FEA57FE4F208130E0092E78
:1010000002C0369527950A94E2F721703327042E03
:1010100001C0220F0A94EAF7822B4F5F5F4F4530E1
:10102000510531F70895BF92CF92DF92EF92FF9270
:101030000F931F93CF93DF938C01C0909001D090BA
:101040009101E0909201F090930180919401909130
:101050009501A0919601B0919701C82AD92AEA2A50
:10106000FB2ACFE1D0E0D701C6010C2E04C0B69513
:10107000A795979587950A94D2F780FD04C021978C
:1010800090F7B12C07C0BC2EB8018C2F0E94470FDF
:101090000197A9F38B2DDF91CF911F910F91FF90B5
:1010A000EF90DF90CF90BF900895CF93DF93EC0146
:1010B0000E941308BE010E94470FDF91CF9108954F
:1010C0001F93CF93DF93EB0190918501992321F03A
:1010D000CB010E94550813C0882349F0CB010E9420
:1010E0001308182F682FCE010E94BA0704C0CB0145
:1010F0000E94E607182FBE01812F0E94470FDF9143
:10110000CF911F9108951F93CF93DF93C0919801C2
:1011100016E080919901C81799F0D0E01C9FF0016A
:101120001D9FF00D1124E656FE4F408151816281D2
:101130007381848195810E949A062196C770E9CFB8
:10114000DF91CF911F9108954091CA015091CB0139
:101150006091CC017091CD018091CE019091CF0131
:101160000C949A06EF92FF920F931F93CF93DF9305
:101170008091CF0182958F7009F065C08091CC017C
:10118000882309F460C080919801F0909901109132
:10119000CA010091CB016091CD017091CE0191E027
:1011A0001F3F09F090E0C0910001D0910101292F6B
:1011B00096E0E92E8F1509F446C06115710521F0FE
:1011C0000F3F21F030E003C031E001C0322F90E04A
:1011D00030FD36C0E89EF001E99EF00D1124DF01DC
:1011E000A656BE4F11963C911197301329C03C91E1
:1011F000311326C012963C911297311121C01396DB
:101200004D915C911497461B570B4C175D07C0F42A
:101210008091CF018F7080618093CF01E156FE4FA6
:1012200080818F70806180838AEC91E00E94180633
:10123000DF91CF911F910F91FF90EF900C94830855
:1012400001968770B7CFDF91CF911F910F91FF90DB
:10125000EF9008959F92AF92BF92CF92DF92EF925C
:10126000FF920F931F93CF93DF93CDB7DEB76197B4
:101270000FB6F894DEBF0FBECDBF8C0185E0F8013C
:10128000DE011D9601900D928A95E1F7D801129624
:10129000EC909091CA01E091CB012091CD01309169
:1012A000CE012115310531F0EF3F31F481E09F3F50
:1012B00019F403C081E001C080E0B82FB1709B2E0B
:1012C00080FD47C1D8014C9111965C9111971396FE
:1012D000AD90BC9014978AECC82E81E0D82EF09087
:1012E000CC01B501621B730B20910001309101010B
:1012F000FF2009F4D9C08091CF016217730708F06D
:1013000095C0282F207F09F052C05E1313C04913E7
:1013100011C0FE2CE1100EC08F7080618093CF0150
:101320000E94A408C6010E9418068091CF01F8010E
:1013300085834DC1AB2831F05F3F31F481E04F3FF1
:1013400019F403C081E001C080E080FD03C081E0AA
:101350008E2502C080E090E0F82FF170FF2E80FF14
:101360001CC0809198012091990136E0821709F400
:101370000BC190E0389FF001399FF00D1124E65623
:10138000FE4F6181561306C06081461303C062811F
:10139000E61203C001968770E9CFFE2CEE2009F417
:1013A00016C18091CF0181608093CF0154C05E133C
:1013B00006C0491304C0E11002C0F80199C0C80179
:1013C0000E948306882361F1EE2051F12091CF0124
:1013D000822F82958F7090E0029774F08091CA01FD
:1013E0009091CB0198878F831986BB86AA862C871C
:1013F000CE0107960E94180686E0F801AAECB1E03B
:1014000001900D928A95E1F70E94B2080E94A4080B
:101410000AC05E1711F1C8010E94830681112CC019
:10142000C8010E941806FF24F394D1C0282F207F02
:1014300081F77A2DB98AA88A6E2D89890E948B0638
:101440008AEC91E00E94180686E0D6011D928A95EA
:10145000E9F70E94A408F12CBAC04913DCCFE110CF
:10146000DACFF8018583C8010E94180686E0D6010C
:101470001D928A95E9F7ABC0EE2091F22091CF0141
:10148000822F82958F7090E002970CF4B5CF8091F7
:10149000CA019091CB019A8389831B82BD82AC8261
:1014A0002E83CE010196A6CF6217730708F044C0C1
:1014B000FE2CEE2009F4B4CF5E1330C049132EC0C9
:1014C0002091CF0120FD21C0822F82958F70482F5F
:1014D00050E041155105C9F0F80125834F30510501
:1014E00041F08F5F982F9295907F822F8F70892B7C
:1014F0008583C8010E94180686E0F801AAECB1E0D5
:1015000001900D928A95E1F73CC086E0F801AAECC3
:10151000B1E001900D928A95E1F759C0C8010E948F
:101520008306811169CF8091CF0181608093CF01C3
:10153000C8010E9418064BC07A2DB98AA88A6E2D60
:1015400089890E948B0686E0D6011D928A95E9F76B
:1015500018C0EE2009F464CFC8010E948306F82E5B
:10156000882309F45DCF86E0F801AAECB1E0019090
:101570000D928A95E1F78AEC91E00E9489020E941F
:10158000B2080E94A40823C04D875E878D859E8582
:101590000E945508292F22952F70223028F49F7021
:1015A00039F0811105C00BC0243028F49F7049F434
:1015B000805E883020F0C8010E9418069F2CF92C0C
:1015C00006C0D80115969C91907F91F7F8CF8F2D8A
:1015D00061960FB6F894DEBF0FBECDBFDF91CF91FD
:1015E0001F910F91FF90EF90DF90CF90BF90AF9041
:1015F0009F9008951F93CF93DF93CDB7DEB72C97BD
:101600000FB6F894DEBF0FBECDBF4F8358876987F2
:101610007A878B879C87CE0107960E942A098823A8
:10162000D1F09F8188852A853B85232B31F08F3F20
:1016300031F481E09F3F19F403C081E001C080E0F4
:1016400080FD47C04F81588569857A858B859C854B
:101650000E949A063EC086E0FE013796DE01119692
:1016600001900D928A95E1F7FF81E8856A857B8577
:101670006115710531F0EF3F31F481E0FF3F19F45E
:1016800003C081E001C080E080FD23C0209199016A
:1016900030E0C9010196877099274091980150E088
:1016A00084179507F1F1F983EA837D836C8396E0D3
:1016B000929FD001939FB00D1124A656BE4FFE01FC
:1016C000319601900D929A95E1F7809399010E94CD
:1016D000830816E08091980190919901891771F122
:1016E000189FC001112486569E4F0E942A09882304
:1016F00029F1E09198011E9FF0011124E656FE4F5A
:101700004081518162817381848195810E949A0612
:101710008091980190E001968770992780939801B5
:10172000D9CF0E9464061092990110929801EAECB8
:10173000F1E086E0DF011D928A95E9F72C960FB65D
:10174000F894DEBF0FBECDBFDF91CF911F910895FA
:101750008091F00185958595859508958091F0019A
:10176000877008959091F001977081E009F480E00E
:10177000089580911302089590911302892B80930C
:101780001302089580959091130289238093130288
:10179000089510921302089590911202892B80935C
:1017A000120208958095909112028923809312026B
:1017B00008951092120208958091F10108950895FC
:1017C0000C94DF0B0C94E00B9091610292FD08C029
:1017D0009091F101981721F08093F1010C94E20BA4
:1017E00008958091F101882329F01092F10180E0A1
:1017F0000C94E20B0895CF93DF93E0910201F091F6
:101800000301809113028083E0910201F0910301B2
:10181000908180911202892B80838091F10188232D
:1018200081F0E0910201F09103019081892B808386
:1018300080910201909103010E94D01681110E94B3
:10184000F10BC0910201D091030140E250E060ED44
:1018500071E0CE010E94981F892B69F080E2FE01A1
:10186000A0EDB1E001900D928A95E1F7CE01DF91F4
:10187000CF910C947C16DF91CF9108950C94DF0BDF
:101880009091610292FD10C098E0899F900111240F
:10189000262B2093F0010E941C078091F001859572
:1018A000859585950C943E0C0C941C071092F001C4
:1018B00080E00C943E0C2091F0018095822380936F
:1018C000F001982F977099F430E0482F082E000C03
:1018D000550B2417350759F09091610292FD07C00E
:1018E0008595859585950E943D070C94560C089525
:1018F0009091610292FB222720F9281769F080FB62
:1019000092F99093610280916002909161020E942D
:10191000C60C82E00C945B0C08958091610282FBFE
:10192000882780F991E089270C94780C81E00C9449
:10193000780C80E00C94780C6FEF7FEF80E090E003
:101940000C94D11F80E090E00E94AD1F21E0893E01
:101950009E4F09F020E0822F089582E090E00C94E1
:10196000A51F83E090E00C94A51FCF9384E090E046
:101970000E94A51FC82F82E290E00E94A51F2C2F75
:1019800030E0A901582BCA01CF910895CF93C92FF8
:10199000682F84E090E00E94B31F6C2F82E290E0F9
:1019A000CF910C94B31FAB01BC018FE090E00C947D
:1019B000C51FAB01BC0183E190E00C94C51F60E042
:1019C00070E0CB010C94D90C60E070E0CB010E9478
:1019D000D30C0C94DF0C69EE7EEF80E090E00E9467
:1019E000D11F60E082E090E00E94B31F60E083E0DE
:1019F00090E00E94B31F10929401109295011092F2
:101A000096011092970160E084E090E00E94B31F7D
:101A100060E082E290E00E94B31F60E085E090E029
:101A20000E94B31F60E086E090E00E94B31F6FEF5A
:101A300087E090E00E94B31F40E050E0BA0188E0E8
:101A400090E00E94C51F60E08DE090E00E94B31F0F
:101A500040E050E0BA0188E190E00E94C51F60E0DC
:101A600087E190E00E94B31F40E050E0BA018CE1B2
:101A700090E00E94C51F60E070E080E290E00E946C
:101A8000D11F40E050E0BA0188E190E00E94C51FFC
:101A90000C94E40C0C94EB0C682F8EE090E00C940A
:101AA000B31F0E94371860931A0270931B02809331
:101AB0001C0290931D02609316027093170280938C
:101AC000180290931902089585B7806885BF85B77D
:101AD000806885BF089581E008950C946B0D08958A
:101AE0000C946F0D0C946F0D0C94720D0C946F0D83
:101AF0000C94760D0C946F0D0E94640D83E290E1BE
:101B00000E9466160E947A0D0C94780D0E94700D4A
:101B10000C946F0D0E943D100C9423020E94221819
:101B20000E9408110E948A0D0C94740D8F929F924E
:101B3000AF92BF92CF92DF92EF92FF920F931F93DB
:101B4000CF93DF93CDB7DEB72A970FB6F894DEBFF9
:101B50000FBECDBF0E941711982E81110E94510D0A
:101B600084E1A82E82E0B82E00E010E0802E802FC5
:101B70000E946110D82EF501C1905F01C826B1F412
:101B80000F5F1F4F0230110589F78FEF89838A831A
:101B90001B820E942B188160782F9D838C83498142
:101BA0005A816B818D810E943F022FC080911E025D
:101BB00081FD0E946710E12CFF24F3948C2D8F216E
:101BC000F1F00E946D0D882399F0EE828F82DF2064
:101BD00081E009F480E088870E942B188160782FCB
:101BE0009A8789874E815F8168858A850E943F0236
:101BF000F801EC5EFD4F8081F826F08206C0E39488
:101C0000FF0CF5E0EF12DACFBBCF81E0911001C0FD
:101C100080E02A960FB6F894DEBF0FBECDBFDF91ED
:101C2000CF911F910F91FF90EF90DF90CF90BF90D9
:101C3000AF909F908F9008950E94960D0E94071379
:101C40000C943402CF93DF930E944C0FEC0181156A
:101C500021E5920708F045C0811530E5930708F0AB
:101C600094C0883E910528F5803E910508F0F8C0A3
:101C7000883A910570F4853A910508F07CC081306E
:101C8000910509F475C008F4E8C0049708F0E8C0AD
:101C9000E4C08F3B910508F0E0C0C85AD0E0CC0FFB
:101CA000DD1FC65BDE4F0990D881C02DCE01946444
:101CB000D8C0811540E2940758F4811551E095078A
:101CC00008F0CEC08D3E910508F4C7C09065C9C02C
:101CD000C11580E4D80708F4C0C0DF70CE01906A57
:101CE000C0C0811525E59207A8F4811534E5930756
:101CF00008F095C0811543E5940708F07BC0811575
:101D000052E5950708F061C0D82FCC27CE01816F2E
:101D1000906AA7C0C11589E5D807A0F4C11528E5C8
:101D2000D20708F082C0C11536E5D30708F095C088
:101D30008C2F0E94E00F8F7190E0D82FCC27CE011E
:101D400090628FC0C1154AE5D40708F474C0CE0173
:101D500090568115904208F080C08D2F8F710E949F
:101D6000E00FDD27D0628F71AE01582BCA0179C018
:101D700081E090E076C0C55AD0E0C858DE4F888137
:101D8000C82FD0E0CE0190646CC074E09695879522
:101D90007A95E1F7282F23703C2F337081E090E093
:101DA00002C0880F991F3A95E2F79C68AC01522B4C
:101DB0009A019C2F9F709695969550E2959FE00111
:101DC0001124C9018C2B9D2B4CC08370992721E0D5
:101DD00030E002C0220F331F8A95E2F79C2F9695C0
:101DE000969580E2989FE0011124C22BD32BCE015F
:101DF0009C6837C08370992721E030E002C0220F31
:101E0000331F8A95E2F79C2F9695969540E2949F12
:101E1000E0011124C22BD32BCE019A6822C0D82F07
:101E2000CC27CE01846F906A1CC0DC2FCC27CE015A
:101E3000806F906A16C08C2F8F700E94E00F94E024
:101E4000D695C7959A95E1F7CF70D0E0DC2FCC27D7
:101E5000D0699E01282BC90104C080E090E001C038
:101E6000CE01DF91CF9108952AE0829FC001112415
:101E7000FC0125E0729FE00DF11D1124E60FF11D1C
:101E8000EE0FFF1FE852FF4F8591949108950E9435
:101E9000340F0E94220E08958238910569F1B0F442
:101EA0008133910509F46DC048F48932910509F434
:101EB00063C08A32910509F469C00895853391059C
:101EC00009F455C089339105B9F00895833E910511
:101ED00069F138F4803E9105B1F0823E910509F137
:101EE0000895863E9105A9F1873E9105B9F1843E9A
:101EF000910509F064C023C02091600220FD4FC00D
:101F000021FD4DC008958091600280FD44C0809104
:101F1000610280FF44C08091600284FD42C083EE74
:101F20004DC08091600282FF38C0F5CF8091600281
:101F300082FD33C08091610280FD31C0ECCF809181
:101F4000610281FF32C08091600284FD2AC087EE69
:101F500035C08091600283FF26C0F5CF809160027A
:101F600083FD21C08091610281FD1FC0ECCF809173
:101F7000600285FD1CC01DC08091600285FD19C0F6
:101F800016C08091600286FD16C017C08091600265
:101F900086FD13C010C089E311C082EE0FC080EE31
:101FA0000DC080E00BC086EE09C084EE07C089E258
:101FB00005C085E303C08AE201C081E390E0089593
:101FC0009091600292FF0DC0282F2871283019F4DB
:101FD000877F846006C0282F2471243011F48B7F02
:101FE000886093FF0DC0282F2871283119F4877E4F
:101FF000846106C0282F2471243111F48B7E8861FE
:102000002091610220FF0DC0382F3871383019F44B
:10201000877F816006C0382F3171313011F48E7F97
:10202000886021FF0DC0282F2871283119F4877E80
:10203000816106C0282F2171213111F48E7E8861C3
:1020400094FD877E089580E008950C949C0C0E9476
:1020500017118FE39CE90197F1F700C000000E947F
:10206000171180E00E94611080FF04C00E942510BB
:102070000C94781808950C9427100E94A20C8111DA
:1020800002C00E944A0D0E94AD0C80931E020E9465
:10209000B50C90936102809360020E943B100E94F5
:1020A000B10C682F70E080E090E00E94BC06609167
:1020B00090017091910180919201909193010C9403
:1020C000F406E82FF0E0EC59FD4F80810895089563
:1020D00080EA8A95F1F7089500C008950C9468107D
:1020E00008950C9470100C9471100C947010F89466
:1020F000E82FE295EF70F0E031A1282F2F7081E0FA
:1021000090E001C0880F2A95EAF7982F90959323C5
:1021100091A392A1892B82A378940895CF93DF9302
:1021200083E30E94771082E30E947710CBE7D1E02F
:1021300089918F3F11F00E94771081E0C038D80755
:10214000B9F7DF91CF910895CF92DF92EF92FF928E
:102150000F931F93CF93DF938C01C62FD0E0CE0156
:1021600080589E4F7C01FC0190819F3F09F447C03D
:10217000D62EF894E92FE295EF70F0E081A19F70E0
:1021800021E030E001C0220F9A95EAF7822B81A36B
:1021900082A12095282322A378940E946C10EBE75B
:1021A000F1E040E851E031E0C12C21912F3F89F06E
:1021B000A22FA295AF70B0E090968C9190E02F7016
:1021C00002C0959587952A95E2F780FD02C0832F7E
:1021D00001C080E0C82A330F4E175F0731F7F701BF
:1021E00080818F3F11F00E94771061E0C11001C023
:1021F00060E08D2D0E946E10C00FD11FC882DF914C
:10220000CF911F910F91FF90EF90DF90CF900895A5
:102210000E948E1010926502109264021092630266
:102220001092620282E00E944F110C94AE011F9343
:10223000CF93DF9300D0CDB7DEB71A82198260E06A
:10224000CE0101960E94A41061E0CE0101960E9489
:10225000A41042E050E0BE016F5F7F4F82E692E043
:102260000E94981F11E0009709F410E0892B31F0CB
:1022700089819A819093630280936202212F42E0C8
:1022800064E672E082E692E00E9450110E94B00182
:10229000812F0F900F90DF91CF911F910895089596
:1022A000FF920F931F93CF93DF938C01F62ED72FBE
:1022B000C42F222349F081E0809321020E942B1831
:1022C0009093200280931F02809121028823C1F005
:1022D00080911F02909120020E944318059780F080
:1022E000EF2DFD2FD8014C2F50E0CD01801B910B1D
:1022F000841795071CF48D918193F7CF10922102DA
:10230000DF91CF911F910F91FF9008950E94301A95
:102310000E948E0D0C943C1A0E94401A0E941C0EC2
:102320000C945A1A0E94C9170E94171A0E947C0D19
:102330000E9486110E948C110E94860DFBCF809115
:10234000280280FF06C06091090170E0660F771FC8
:1023500026C081FF04C06091090184E005C082FFAE
:1023600007C06091090188E0689FB001112417C07F
:10237000909127029923D1F060910801961788F770
:102380002091090188E0289F90011124929FA001CB
:10239000939F500D112470E0CA010E946A1F60389B
:1023A000710540F46115710519F406C068E070E02C
:1023B000862F08958FE7089581E00895809128027F
:1023C00080FF08C06091050170E07595679575956F
:1023D000679521C081FF06C06091050170E0759589
:1023E000679519C082FF04C06091050170E010C0BC
:1023F00090912602992399F0609104019617A0F715
:1024000080910501899FC001112470E00E946A1F1C
:102410006038710540F46115710519F406C061E07A
:1024200070E0862F08958FE7089581E008958D3E2E
:1024300021F40E949F11819504C08E3E29F40E94D0
:102440009F1180932C0208958F3E21F40E949F11CA
:10245000819504C0803F29F40E949F1180932B0234
:102460000895893F19F40E94DE1105C08A3F31F4B6
:102470000E94DE11819580932D0208958B3F21F4F7
:102480000E94DE11819504C08C3F29F40E94DE1168
:1024900080932E0208959FE0980F983078F421E001
:1024A00030E0A90102C0440F551F9A95E2F7CA0116
:1024B00090912A02892B80932A0208958D3F21F45E
:1024C0008091280281600BC08E3F21F48091280208
:1024D000826005C08F3F29F4809128028460809338
:1024E000280208958D3E39F490912C0297FF35C053
:1024F00010922C0259C08E3E29F490912C0219168C
:10250000BCF32BC090912B028F3E29F497FF25C07E
:1025100010922B0249C0803F19F41916CCF31DC04C
:1025200090912D02893F29F41916BCF410922D02C6
:102530003BC08A3F19F497FF10C0F8CF8B3F39F4A6
:1025400090912E0297FF09C010922E022DC08C3F51
:1025500021F490912E021916BCF39FE0980F983049
:1025600080F421E030E0A90102C0440F551F9A9584
:10257000E2F7CA01809590912A02892380932A026A
:1025800013C08D3F21F4809128028E7F0BC08E3FB7
:1025900021F4809128028D7F05C08F3F29F480911E
:1025A00028028B7F8093280280912B02811106C024
:1025B00080912C02811102C01092270280912D027D
:1025C000811106C080912E02811102C01092260254
:1025D00008950E942B1820912B02211104C02091F4
:1025E0002C02222321F09093250280932402209133
:1025F0002D02211104C020912E02222321F090935C
:1026000023028093220289E292E00C949616EF92C4
:10261000FF920F931F93CF93DF9300D000D000D091
:10262000CDB7DEB786E0E9E2F2E0DE011196019077
:102630000D928A95E1F7E0902B02F0902C02009128
:102640002D0210912E0210922B0210922C02109249
:102650002D0210922E02E11003C0FF2009F45DC08C
:1026600080912402909125020E944318AC01909120
:102670002702992339F020910A0130E02417350709
:1026800058F04BC020910B018AE0289F9001112443
:102690002417350718F041C09F3F19F09F5F9093B2
:1026A0002702EE2061F00E949F111E1414F09FEF8C
:1026B00001C091E0989F902D112490932B02FF2050
:1026C00061F00E949F111F1414F09FEF01C091E070
:1026D000989F902D112490932C0230912B0233233C
:1026E000E1F020912C022223C1F045EB3403C0011C
:1026F0001124992319F090932B0203C081E0809359
:102700002B0235EB2303C0011124992319F0909378
:102710002C0203C081E080932C02011103C011231D
:1027200009F45DC080912202909123020E94431817
:10273000AC0190912602992339F02091060130E0F6
:102740002417350758F04BC0209107018AE0289FD5
:10275000900111242417350718F041C09F3F19F04C
:102760009F5F90932602002361F00E94DE111016F5
:1027700014F09FEF01C091E0989F902D1124909349
:102780002D02112361F00E94DE11111614F09FEF4B
:1027900001C091E0989F902D112490932E023091CA
:1027A0002D023323E1F020912E022223C1F045EBCC
:1027B0003403C0011124992319F090932D0203C012
:1027C00081E080932D0235EB2303C001112499236E
:1027D00019F090932E0203C081E080932E02809125
:1027E0002B0281110BC080912C02811107C08091B6
:1027F0002D02811103C080912E0281110E94E912E5
:10280000EB82FC820D831E8386E0FE013196A9E2F5
:10281000B2E001900D928A95E1F726960FB6F894F2
:10282000DEBF0FBECDBFDF91CF911F910F91FF9003
:10283000EF900895E9E2F2E086E0DF011D928A95CB
:10284000E9F71092270210922602109228020895AA
:10285000CF93DF93EC01FB018281882309F43CC113
:10286000C430FDE5DF0760F4CB3F9CE5D90788F471
:102870009E0122503C452431310508F02EC109C08B
:10288000C236EDE5DE0729F0C63AFDE5DF0709F0BF
:1028900024C10E94B50C9093610280936002C13103
:1028A0008CE5D80709F4C6C008F042C0C930ECE591
:1028B000DE0709F49BC000F5C5308CE5D80709F4A4
:1028C00085C078F4C330ECE5DE0709F478C008F081
:1028D0007AC0C230DC4509F0F5C0809160028160A9
:1028E000EFC0C7309CE5D90709F478C008F07AC07A
:1028F000809160028061E4C0CD30FCE5DF0709F41F
:1029000087C058F4CB309CE5D90709F479C008F0AA
:102910007BC08091600288606FC0CF30FCE5DF072C
:1029200009F480C008F082C080916002877FC8C02F
:10293000CE3F9CE5D90709F471C000F5C531FCE52F
:10294000DF0709F485C068F4C3319CE5D90709F4B1
:1029500075C008F095C00E946406809160028F7770
:10296000AFC0CC3FFCE5DF07A9F108F054C0CB3F76
:10297000DC4509F0A7C08091610240C0C230EDE59E
:10298000DE0709F489C058F4C1158DE5D80709F4AC
:102990005AC008F069C08091610282602FC0C236BF
:1029A000EDE5DE0709F47CC0C63AFDE5DF0709F472
:1029B00081C0C330DD4509F085C080E06EC08091E4
:1029C000600282607DC08091600216C080916002CA
:1029D000886076C08091610282604FC08091600201
:1029E00080626EC08091600280646AC00E9464064A
:1029F00080916002806864C0846062C081603DC074
:102A0000809160028E7F5CC0809160028D7F58C093
:102A10008091600216C08091610218C080916102AD
:102A20008D7F2BC0809160028F7E4AC080916002B2
:102A30008F7D46C0809160028F7B42C08091600292
:102A4000877F8B7F3DC0809161028D7F8E7F15C017
:102A50008091600282FB222720F991E0922790FB6F
:102A600082F990FB83F92CC080916102982F909598
:102A700091708E7F892B90FB81F98093610222C037
:102A80000E9464068091600287FB222720F991E072
:102A9000922790FB87F914C081E00E944C0D12C070
:102AA0008091600284FB222720F991E0922790FB1D
:102AB00084F906C080916002982F909590FB80F970
:102AC0008093600280916002909161020E94C60C26
:102AD0000E94640680E001C081E0DF91CF910895FB
:102AE000CF93DF9386319C4541F5EB010E94B90BF2
:102AF000982F8A812091020130910301882379F077
:102B00009A7A81E009F480E080932F02911102C04B
:102B100069E201C065E3C9010E9466170AC080919D
:102B20002F02811102C069E201C065E3C9010E9460
:102B300071170E94FB0B80E001C081E0DF91CF9113
:102B400008950F931F93CF93DF93C42FD22FFC01CF
:102B500082818823C9F0409332020E942B189093FF
:102B600031028093300280E28C0F883008F057C029
:102B7000C77081E001C0880FCA95EAF7DF91CF9155
:102B80001F910F910C94C10380913202481330C001
:102B900080913002909131020E9443188A3F910542
:102BA00038F510E21D0FCD17B9F080E28C0F883098
:102BB00040F4C77081E001C0880FCA95EAF70E940F
:102BC000C803183028F581E09D2F977001C0880F49
:102BD0009A95EAF70E94C103802F0E94B80318302B
:102BE000F0F4D77081E001C0880FDA95EAF70AC0E7
:102BF00080E28C0F883098F4C77081E001C0880FA4
:102C0000CA95EAF7DF91CF911F910F910C94C803F9
:102C1000802FDF91CF911F910F910C94B803DF911A
:102C2000CF911F910F9108950F939C01CB01243FE9
:102C30004CE5340731F188F4293DFCE53F07D9F034
:102C40002A3D4CE5340779F1283D3C45A9F506E2DB
:102C500021EE41EE68ED7CE52BC0263FFCE53F0709
:102C6000E1F0A8F0273F3C4539F507E225EE46EEB6
:102C700067EF7CE51DC007E225EE45EE69ED7CE5DA
:102C800017C006E221EE40EE64EF7CE511C007E2DA
:102C900025EE44EE65EF7CE50BC006E221EE42EE48
:102CA00066EF7CE505C008E221E045EE6AED7CE5D3
:102CB0000E94A11580E008C0FC018281882319F0E0
:102CC0001092320201C081E00F9108959093830128
:102CD000809382010895909338028093370208957B
:102CE000E0913702F0913802309721F00190F081A5
:102CF000E02D099480E00895E0913702F0913802C8
:102D0000309799F020911801222359F02091600208
:102D100027FF07C0DC012C9111962C93119726E018
:102D20002C930280F381E02D09940895E0913702FD
:102D3000F0913802309739F022E0DC012C930480C6
:102D4000F581E02D099408952091350230913602E5
:102D50002817390771F09093360280933502E0917D
:102D60003702F0913802309721F00680F781E02D8C
:102D700009940895209133023091340228173907BD
:102D800071F09093340280933302E0913702F09116
:102D90003802309721F00084F185E02D09940895E0
:102DA000FC01329680911801882331F080916002F5
:102DB00087FF02C09EE101C096E080E0915028F0BC
:102DC00021912223D9F38F5FF9CF0895662351F122
:102DD000209118012223E9F02091600227FF19C0F9
:102DE000462F4695469546954E31E0F4677021E0B2
:102DF00030E002C0220F331F6A95E2F7FC01E40FB6
:102E0000F11D828190E02823392381E0232B69F48E
:102E100009C0FC01329608962191621729F0E81743
:102E2000F907D1F780E0089581E008959C01FC0145
:102E300032969FEF80E04191461789F09F3F19F449
:102E4000411101C0982F8F5F8630A9F79F3F39F05D
:102E5000F901E90FF11D97FDFA9562830895089530
:102E60009C012A5F3F4FFC014281461301C0128240
:102E7000019682179307B9F70895262F2695269570
:102E800026952E3168F4FC01E20FF11D677021E0F8
:102E900030E001C0220F6A95EAF78281282B228355
:102EA0000895262F2695269526952E3170F4FC013F
:102EB000E20FF11D677021E030E001C0220F6A953A
:102EC000EAF7209582812823228308952091180112
:102ED000222329F02091600227FD0C943D170C94C9
:102EE000161720911801222329F02091600227FD56
:102EF0000C9451170C94301720911801FC01329654
:102F0000222331F08091600287FF02C08EE101C070
:102F100086E0DF011D928A95E9F7089508950C94E3
:102F20008E1783E0809339020C948F17811102C0B1
:102F300081E001C082E0809339020C948F170C94D9
:102F4000961781E0809339020C948F170C94A11787
:102F500008950C94A8170C94A9170C94A8170C9416
:102F6000A8170C94A8170E94AF170E9417110E946F
:102F7000AD1780E00E946110811108C081E00E94BD
:102F8000611091E0811103C090E001C091E0892FB0
:102F9000089508951F920F920FB60F9211248F93E8
:102FA0009F93AF93BF9380913A02811113C0809198
:102FB000660290916702A0916802B0916902419601
:102FC000A11DB11D8093660290936702A0936802D1
:102FD000B0936902BF91AF919F918F910F900FBEF7
:102FE0000F901F90189580916E02843031F10E94ED
:102FF000140210923A0220E488E190E00FB6F894AF
:10300000A895809360000FBE2093600083B7817FF6
:10301000846083BF83B7816083BF7894889583B7CA
:103020008E7F83BF0FB6F894A89580916000886169
:1030300080936000109260000FBE08950E946406A5
:103040000C94180282E084BD93E095BD9AEF97BD81
:1030500080936E0008952FB7F89480916602909146
:103060006702A0916802B09169022FBF08952FB73F
:10307000F894609166027091670280916802909165
:1030800069022FBF08959C014FB7F89480916602A2
:1030900090916702A0916802B09169024FBF821BB4
:1030A000930B089578941F920F920FB60F921124EC
:1030B0008F939F93AF93BF93809166029091670225
:1030C000A0916802B09169020196A11DB11D809383
:1030D000660290936702A0936802B0936902BF9161
:1030E000AF919F918F910F900FBE0F901F901895E9
:1030F00087E797E790930108809300089AE088E1BA
:103100000FB6F894A895809360000FBE909360006E
:10311000FFCF80915E020895089522E02093E90098
:103120002FEF3091E800215035FD06C035ED3A957E
:10313000F1F700002111F5CF2091E80025FF0BC029
:1031400040E050E066E070E00E94CC1A8091E80018
:103150008E778093E8000895CF93DF932091180134
:10316000222339F02091600227FF03C060E222E0B1
:1031700002C068E021E02093E9002FEF3091E800E1
:10318000215035FD06C035ED3A95F1F700002111CB
:10319000F5CF2091E80025FF1DC0EC0180911801BA
:1031A000811105C040E050E068E070E003C070E0CD
:1031B00040E050E0CE010E94CC1A8091E8008E776A
:1031C0008093E80080E2FE01AEE3B2E001900D9250
:1031D0008A95E1F7DF91CF91089580933B02709338
:1031E0003D0260933C0280916E02843001F582E0E2
:1031F0008093E9008FEF9091E800815095FD06C023
:1032000095ED9A95F1F700008111F5CF8091E800D6
:1032100085FF0DC040E050E063E070E08BE392E09A
:103220000E94CC1A8091E8008E778093E800089580
:10323000BC0184E00C94ED18BC0183E00C94ED1803
:1032400080916D02811109C00E945D1C0E94BA1C10
:103250008091E20084608093E200089510926D02F4
:1032600008950C94A61760916A0281E0611101C073
:1032700080E00C94911790916E0281E0943009F0F7
:1032800080E060916A020C94961742E061EC81E064
:103290000E94D61B42E261EC82E00E94D61B909114
:1032A0006E0281E0943009F080E060916A020C9433
:1032B0009F1780917002833009F461C030F481302F
:1032C00071F0823009F49AC008958A3009F486C0FA
:1032D0008B3009F46CC0893009F0A8C020C08091FF
:1032E0006F02813A09F0A2C08091E800877F809345
:1032F000E8008091730290917402892B21F460E2BE
:103300008EE392E003C060E080E090E070E00E9415
:10331000171B8091E8008B778093E80008958091D7
:103320006F02813209F082C0809173029091740221
:10333000029708F07BC08091E800877F8093E800C7
:103340008091E80082FD05C080916E028111F8CF66
:103350006DC02091F3008091F20090E0922B0297D3
:1033600031F48091F100813011F0863021F48091A8
:10337000F10080935E028091E8008B7753C08091CA
:103380006F02813A09F052C08091730290917402E9
:10339000892B09F04BC08091E800877F8093E8007B
:1033A0008091E80080FFFCCF8091180136C08091A9
:1033B0006F028132D9F58091730290917402892B4A
:1033C000A9F58091E800877F8093E8000E940B1C9C
:1033D00080917102809318010C94640680916F02B1
:1033E000813221F58091E800877F8093E8000E9478
:1033F0000B1C8091720280935F02089580916F028E
:10340000813AA1F48091E800877F8093E800809161
:10341000E80080FFFCCF80915F028093F1008091F3
:10342000E8008E778093E8000C940B1C089584B715
:10343000877F84BF0FB6F894A8958091600088615B
:1034400080936000109260000FBE90E080E80FB69D
:10345000F89480936100909361000FBE0C94A117C3
:103460000E945D1C0E94BA1CE2EEF0E08081846044
:10347000808378940C944F1F8CE091E00C946B1631
:1034800080916E028530A9F480916E02853079F4C6
:103490000E94F31780916C028823B1F30E94B31746
:1034A000882391F30E94B61A0E946406EDCF0C9413
:1034B0001E18089508950C945D1A292F3327233080
:1034C0003105C9F060F42130310581F02230310539
:1034D00009F044C08BE390E02AE231E043C021329E
:1034E0003105E1F02232310549F138C082E190E046
:1034F00025E631E037C099278130910549F028F061
:10350000029761F5ECEEF0E005C0E6E2F1E002C002
:10351000E2E0F1E0849190E09F0124C06115710523
:1035200041F061307105D1F489E090E025E531E0AA
:1035300019C089E090E02CE331E014C061157105F9
:1035400041F06130710551F486EB90E027E731E0FE
:1035500009C080E490E02DE232E004C080E090E019
:1035600020E030E0FA0131832083089580E189BDB5
:1035700082E189BD09B400FEFDCF8091D8008F7D26
:103580008093D8008091E00082608093E000809179
:10359000E00081FDFCCF0895CF92DF92EF92FF9281
:1035A0000F931F93CF93DF93EC018B017A010E945D
:1035B0002A1C811133C0E114F10439F0F701808134
:1035C0009181081B190BC80FD91FC12CD12C0115D3
:1035D000110519F18091E80085FD16C08091E80081
:1035E0008E778093E800E114F10449F0F7018081BF
:1035F0009181C80ED91ED182C08285E00FC00E9481
:103600002A1C882321F30AC089918093F10001507C
:103610001109FFEFCF1ADF0ADACF80E0DF91CF91F7
:103620001F910F91FF90EF90DF90CF900895209120
:103630007502309176022617370748F0611571053B
:1036400039F42091E8002E772093E80001C0B901F9
:10365000FC0120E06115710579F180916E028823EB
:10366000F1F18530F1F18091E80083FD3CC080915B
:10367000E80082FD2EC08091E80080FFEBCF209112
:10368000F3008091F20090E0922B6115710551F0EA
:103690008830910538F421912093F100615071092F
:1036A0000196F3CF21E0089709F020E08091E8002F
:1036B0008E778093E800CECF2111CFCF0AC08091C2
:1036C0006E02882361F0853061F08091E80083FD0F
:1036D0000AC08091E80082FFF2CF80E0089582E086
:1036E000089583E0089581E0089520917502309156
:1036F00076022617370748F06115710539F42091D5
:10370000E8002E772093E80001C0B901FC0120E019
:103710006115710591F180916E02882309F440C012
:10372000853009F43FC08091E80083FD3DC0809161
:10373000E80082FD2FC08091E80080FFE9CF209152
:10374000F3008091F20090E0922B6115710559F021
:103750008830910540F424912093F1003196615016
:1037600071090196F2CF21E0089709F020E08091DD
:10377000E8008E778093E800CBCF2111CCCF0AC030
:1037800080916E02882361F0853061F08091E800BD
:1037900083FD0AC08091E80082FFF2CF80E00895A7
:1037A00082E0089583E0089581E00895982F97308E
:1037B00068F59093E900981739F07091EC0020912A
:1037C000ED005091F00003C0242F762F50E021FD32
:1037D00002C09F5FECCF3091EB003E7F3093EB0057
:1037E0003091ED003D7F3093ED003091EB00316082
:1037F0003093EB007093EC002093ED005093F000B9
:103800002091EE0027FDE5CF80E008958F70809332
:10381000E90081E0089580916F0287FF11C08091D7
:10382000E80082FD05C080916E028111F8CF11C0C1
:103830008091E8008B770BC080916E02882349F05D
:103840008091E80080FFF8CF8091E8008E77809328
:10385000E80008952091E4003091E50095E640915C
:10386000EC00842F817040FF23C08091E80080FD30
:103870001DC080916E02882399F0853099F0809167
:10388000EB0085FD11C04091E4005091E500241744
:10389000350729F3915011F09A01E1CF84E00895A2
:1038A00082E0089583E0089581E0089580E008951E
:1038B0004091E80042FFDDCF08950E94CB1C0E949A
:1038C000D31CE0EEF0E0808181608083E8EDF0E0E1
:1038D00080818F77808319BCA7EDB0E08C918E7FBB
:1038E0008C9380818F7E808310926D0208950F9358
:1038F0001F93CF93DF930E94CB1C0E94D31CC8ED73
:10390000D0E088818F7788838881806888838881E8
:103910008F7D888319BC10926E0210926A021092F9
:103920006C0210926B0200EE10E0F80180818B7F38
:10393000808388818160888342E060E080E00E942B
:10394000D61BE1EEF0E080818E7F8083E2EEF0E036
:10395000808181608083808188608083F80180819C
:103960008E7F8083888180618883DF91CF911F91D2
:103970000F910895E8EDF0E080818F7E8083E7ED80
:10398000F0E080818160808384E082BF81E0809369
:103990006D020C94771CE8EDF0E080818E7F8083CF
:1039A0001092E20008951092DA001092E10008955A
:1039B0001F920F920FB60F9211242F933F934F93A4
:1039C0005F936F937F938F939F93AF93BF93EF9387
:1039D000FF938091E10082FF0BC08091E20082FFA3
:1039E00007C08091E1008B7F8093E1000E944E1F11
:1039F0008091DA0080FF1FC08091D80080FF1BC03B
:103A00008091DA008E7F8093DA008091D90080FF68
:103A10000DC080E189BD82E189BD09B400FEFDCF02
:103A200081E080936E020E94201905C019BC10929B
:103A30006E020E942E198091E10080FF19C08091D2
:103A4000E20080FF15C08091E2008E7F8093E2004B
:103A50008091E20080618093E2008091D8008062D2
:103A60008093D80019BC85E080936E020E943319C0
:103A70008091E10084FF30C08091E20084FF2CC07F
:103A800080E189BD82E189BD09B400FEFDCF80914E
:103A9000D8008F7D8093D8008091E1008F7E809345
:103AA000E1008091E2008F7E8093E2008091E2004D
:103AB00081608093E20080916A02882311F084E0A3
:103AC00007C08091E30087FD02C081E001C083E070
:103AD00080936E020E943B198091E10083FF29C010
:103AE0008091E20083FF25C08091E100877F809371
:103AF000E10082E080936E0210926A028091E10000
:103B00008E7F8093E1008091E2008E7F8093E200BF
:103B10008091E20080618093E20042E060E080E01A
:103B20000E94D61B8091F00088608093F0000E9474
:103B30003119FF91EF91BF91AF919F918F917F913B
:103B40006F915F914F913F912F910F900FBE0F900A
:103B50001F9018951F920F920FB60F9211242F935A
:103B60003F934F935F936F937F938F939F93AF9305
:103B7000BF93CF93DF93EF93FF93C091E900CF7092
:103B80008091EC00D82FD17080FDD0E81092E90030
:103B90008091F000877F8093F00078940E94EE1D62
:103BA0001092E9008091F00088608093F000CD2BA6
:103BB000CF70C093E900FF91EF91DF91CF91BF915A
:103BC000AF919F918F917F916F915F914F913F91B5
:103BD0002F910F900FBE0F901F9018951F93CF93AA
:103BE000DF93CDB7DEB7AA970FB6F894DEBF0FBE4E
:103BF000CDBFEFE6F2E08091F100819322E0E7375C
:103C0000F207C9F70E9459198091E80083FF2EC17D
:103C100080916F0290917002492F50E04A30510517
:103C200008F024C1FA01EE59FF4F0C947E1F803832
:103C300021F0823809F01AC108C080916B0290917E
:103C40006C02992389F082600FC0809173028F709B
:103C5000873008F00BC18093E9008091EB0085FB71
:103C6000882780F91092E9009091E800977F90935F
:103C7000E8008093F1001092F100D1C0282F2D7F31
:103C800009F0F4C0882319F0823061F0EFC0809110
:103C90007102813009F0EAC0933009F080E080932E
:103CA0006C022EC08091710281112AC08091730232
:103CB0008F702FEF280F263008F0D8C08093E900CE
:103CC0002091EB0020FF1CC0933021F48091EB0089
:103CD000806214C09091EB0090619093EB0021E022
:103CE00030E0A90102C0440F551F8A95E2F74093C6
:103CF000EA001092EA008091EB0088608093EB006C
:103D00001092E9008091E800877F8093E8000E948C
:103D10000B1CACC08111AAC0109171021F77809159
:103D2000E3008078812B8093E3008091E800877F17
:103D30008093E8000E940B1C8091E80080FFFCCF7C
:103D40008091E30080688093E300111102C082E05B
:103D500001C083E080936E0289C08058823008F0F1
:103D600085C080917102909172028C3D53E095075D
:103D700079F583E08A838AE289834FB7F894DE017C
:103D8000139620E03EE051E2E32FF0E0509357001D
:103D9000E49120FF03C0E295EF703F5FEF708E2F3C
:103DA00090E0EA3010F0C79601C0C0968D939D93C5
:103DB0002F5F243149F74FBF8091E800877F8093C0
:103DC000E8006AE270E0CE0101960E94171B16C05F
:103DD0006091730270917402AE014F5F5F4F0E9459
:103DE0005B1ABC01892B09F441C09091E800977FD0
:103DF0009093E80089819A810E94751B8091E80068
:103E00008B778093E80032C0803881F58091E8009C
:103E1000877F8093E80080916A028093F10080910F
:103E2000E8008E7772CF811121C08091710290914C
:103E3000720299270297D4F48091E800877F8093DB
:103E4000E8008091710280936A020E940B1C8091AD
:103E50006A02811106C08091E30087FD02C081E003
:103E600001C084E080936E020E9445198091E800B1
:103E700083FF0AC08091E800877F8093E8008091EB
:103E8000EB0080628093EB00AA960FB6F894DEBF39
:103E90000FBECDBFDF91CF911F9108950895CF93AD
:103EA00080916E028823A1F0C091E900CF709091BB
:103EB000EC00892F817090FD80E8C82B1092E900FA
:103EC0008091E80083FD0E94EE1DCF70C093E90051
:103ED000CF91089597FB072E16F4009407D077FD35
:103EE00009D00E94841F07FC05D03EF4909581956F
:103EF0009F4F0895709561957F4F0895EE0FFF1FB6
:103F00000590F491E02D0994AA1BBB1B51E107C059
:103F1000AA1FBB1FA617B70710F0A61BB70B881F59
:103F2000991F5A95A9F780959095BC01CD010895E8
:103F3000FB01DC0104C08D910190801921F44150F6
:103F40005040C8F7881B990B0895F999FECF92BD90
:103F500081BDF89A992780B50895A8E1B0E042E0C4
:103F600050E00C94D91F262FF999FECF92BD81BD48
:103F7000F89A019700B4021639F01FBA20BD0FB6A7
:103F8000F894FA9AF99A0FBE08950396272F0E9483
:103F9000B41F0E94B31F252F0E94B41F242F0C941E
:103FA000B41F0196272F0E94B41F0C94B31FDC018D
:103FB000CB01FC01F999FECF06C0F2BDE1BDF89A34
:103FC000319600B40D9241505040B8F70895F894DE
:023FD000FFCF21
:103FD200FA00F201280850011E0A14018918AC18CF
:103FE2008D181C1918198C1801E200E900EA00B5B5
:103FF20000B600B700CD008301CC008A0192019483
:10400200012102230224022502260227022A02B3E8
:1040120000B4006F007000818283E200E900EA00D0
:10402200B500B600B700CD008301CC008A01920131
:1040320094012102230224022502260227022A02D7
:10404200B300B4006F007000818283946697C63417
:02405200333207
:00000001FF
